:1000000000308A00CC280000831A0A289100030ED1
:1000100092000F2883129100030E920092140A0896
:1000200099008A018313910E040893000C08940030
:100030000D0895000E0896000F089700100898000C
:1000400083128B1E25280B193A28130884001408E4
:100050008C0015088D0016088E0017088F001808F0
:10006000900019088A00120E83008312110E921854
:10007000831609003D3081009B0BC928861C45284A
:1000800083168610831286104928831686108312E1
:100090008614831605148312051850289C1C5228B8
:1000A0000030532801308D000D1858281C10592895
:1000B0001C148316051400308312051C01308D00BA
:1000C0000D1864289C1065289C1400301C18013001
:1000D000A10000301C1E01302105003A03198228BE
:1000E0001C159F0B822805309F001C168316851453
:1000F0008312851C7D289C1582289C1981289C15BB
:1001000082289C119C1D97288316061083120614C2
:10011000831685148312851C9628A00B962814300C
:10012000A0009C1183160610831206109D288316CA
:100130000610831206101430A0001C1DAA281D08EA
:1001400003199E039D0BA9289E08031DA9281C12B4
:100150001C11AE2801309E002C309D008316051422
:1001600083120518B8288316061183120611BC28BD
:1001700083160611831206151C1DC32883168611CB
:1001800083128611C72883168611831286150230C2
:100190009B000B118A11252884011F3083051F3015
:1001A000650000306600FF3086009C118316061043
:1001B000831206109C0101309E002C309D000530FA
:1001C0009F001430A00002309B003D3081000730BA
:1001D0008C008C1DF32807308101813084000008D9
:1001E000C0390F3880006400813084000008C039B5
:1001F0000C0480008B168B178B169A01FE28630067
:02400E00F13F80
:00000001FF
